:100000000C94E6000C94F8000C94F8000C94F800A2
:100010000C94F8000C94F8000C94F8000C94F80080
:100020000C94F8000C94F8000C94F8000C94F80070
:100030000C94F8000C94F8000C94F8000C94F80060
:100040000C94F8000C94F8000C9433060C942906D8
:100050000C941F060C94F8000C94F8000C94F80013
:100060000C94F8000C94F8002AFF2B3C420080AE60
:1000700080D580F180D980F180A8803F80D3800036
:100080008040808D801480A080C880DA80108081BC
:10009000807F8020800280DB802080A280A680AFCD
:1000A000802E801080218000807F80228000800749
:1000B000FFFFFFFFFFFFFFFF0009121B242D363F4C
:1000C00048415A536C657E7719100B023D342F2638
:1000D0005158434A757C676E323B2029161F040D28
:1000E0007A7368615E574C452B2239300F061D1418
:1000F000636A7178474E555C646D767F4049525B08
:100100002C253E3708011A137D746F6659504B42F7
:10011000353C272E1118030A565F444D727B6069E7
:100120001E170C053A3328214F465D546B627970D7
:10013000070E151C232A31384148535A656C777EC7
:1001400009001B122D243F3658514A437C756E67B7
:100150001019020B343D262F737A6168575E454CA7
:100160003B3229201F160D046A6378714E475C5597
:10017000222B3039060F141D252C373E0108131A87
:100180006D647F7649405B523C352E2718110A0377
:10019000747D666F5059424B171E050C333A212867
:1001A0005F564D447B7269600E071C152A23383157
:1001B000464F545D626B70792B3C08008008801FAD
:1001C00080B74055FFFFFFFFFFFFFF0011241FBE58
:1001D000CFEFD4E0DEBFCDBF13E0A0E0B1E001C0BF
:1001E0001D92AF35B107E1F70E9460060C94D90962
:1001F0000C940000582F219898E080E0232D31E0E6
:10020000422F00004150E9F73150D1F7209832E0F9
:10021000422F00004150E9F73150D1F7880F19996A
:100220008160209A31E0422F00004150E9F73150BF
:10023000D1F7915021F7511101C0219A332D91E04E
:10024000232F00002150E9F79150D1F72098332D4A
:1002500093E0232F00002150E9F79150D1F7209A25
:10026000332D91E0232F00002150E9F79150D1F771
:10027000712C612C2198089598E0232D31E0422FB4
:1002800000004150E9F73150D1F787FF02C02198B3
:1002900001C0219A880F31E0422F00004150E9F758
:1002A0003150D1F7209832E0422F00004150E9F759
:1002B0003150D1F7209A915009F72198232D82E0EF
:1002C000922F00009150E9F78150D1F72098232D0B
:1002D00082E0922F00009150E9F78150D1F793B15D
:1002E0009270209A332D81E0232F00002150E9F7EE
:1002F0008150D1F7712C612C81E0911101C080E017
:1003000008952098232D81E0922F00009150E9F765
:100310008150D1F7612C712C21980895219A232DB9
:1003200081E0922F00009150E9F78150D1F7612CC4
:10033000712C209A0895582F519898E080E0232D31
:1003400031E0422F00004150E9F73150D1F7509889
:1003500032E0422F00004150E9F73150D1F7880FC9
:1003600049998160509A31E0422F00004150E9F7ED
:100370003150D1F7915021F7511101C0519A332DCD
:1003800091E0232F00002150E9F79150D1F75098C8
:10039000332D93E0232F00002150E9F79150D1F73E
:1003A000509A332D91E0232F00002150E9F791500E
:1003B000D1F7712C612C5198089598E0232D31E0EC
:1003C000422F00004150E9F73150D1F787FF02C0BA
:1003D000519801C0519A880F31E0422F00004150DE
:1003E000E9F73150D1F7509832E0422F00004150E8
:1003F000E9F73150D1F7509A915009F75198232DD0
:1004000082E0922F00009150E9F78150D1F7509887
:10041000232D82E0922F00009150E9F78150D1F70F
:1004200099B19270509A332D81E0232F0000215012
:10043000E9F78150D1F7712C612C81E0911101C055
:1004400080E008955098232D81E0922F0000915074
:10045000E9F78150D1F7612C712C51980895519A88
:10046000232D81E0922F00009150E9F78150D1F7C0
:10047000612C712C509A089520E030E007C048E0CC
:100480004498449A4150E1F72F5F3F4F28173907AE
:10049000B1F7089588B18F6088B9449887B1807F9B
:1004A00087B981E090E210C0449A0000000000008B
:1004B0000000309904C044980000449A089544987C
:1004C0000000000000000000019771F7F4CF44988D
:1004D0003D9AE0915C03F0E0EE0FFF1FE827E8543F
:1004E000FF4FE491E0935C0398E0449887FF02C0DB
:1004F000459A01C04598880F449A9150B1F73D98AC
:100500000895CF93DF9300D000D0CDB7DEB710921F
:100510005C034C835B836A8379830E9467027981E1
:10052000872F0E9467026A81862F0E9467025B8183
:10053000852F0E9467024C81842F0E946702809160
:100540005C03880F81600E94670244983D9881E0B7
:1005500090E209C0449A0000000000000000359BB2
:1005600004C0449800000197A9F70F900F900F90D6
:100570000F90DF91CF9108953D9897E080E03599F5
:1005800081604498880F449A9150C9F735998160E9
:1005900044980000449A0895E9E4F3E0119283E05E
:1005A000E935F807D9F71092480310925B031092CF
:1005B0005A0381E0809359030895CF93DF9300D0CD
:1005C00000D0CDB7DEB7AB01BC018AB18F608AB96C
:1005D00084E690E049835A836B837C830E943C02CB
:1005E00049815A816B817C81CB01AA27BB27BC0141
:1005F00081E50E94810285E090E00E943C028AB180
:10060000807F8AB90E944A02449A0E94CC0280E00C
:1006100092E090935E0380935D030F900F900F9094
:100620000F90DF91CF910895A8E4B3E09C91E92F5A
:10063000F0E0E75BFC4F80819F5F9F709C93089583
:10064000282F90914803E92FF0E0E75BFC4F808171
:1006500030915903332311F12827A92FAC50AF70E3
:10066000B0E0A75BBC4F3C9132273C93A92FA5502B
:10067000AF70B0E0A75BBC4F3C9132273C93208326
:100680009F5F9F709093480320915A0330915B03C2
:100690002F5F3F4F30935B0320935A030895CF930E
:1006A000C82F97B19F6097B9449898B1907F98B937
:1006B00098B182958F70982B98B90E942003449A24
:1006C00000000000449898B1907F98B998B18C2FA1
:1006D0008F70982B98B90E942003449A0000000064
:1006E000CF91089520915D0330915E03211531056E
:1006F00041F02150310930935E0320935D030C9447
:100700004F030895CF93DF9387B1807F87B94498D3
:100710000000449AD6B1D295D07F8D2F82958F70EC
:100720000E94200344980000449AC6B1CF70CD2B9C
:100730008C2F8F700E94200344988C2FDF91CF91D3
:1007400008950F931F93CF93DF9307C00197909362
:100750005E0380935D030E94820380915D0390910C
:100760005E03009799F710925903C8E0D0E00E9409
:100770008203182F0E941403082F0E94140390E193
:10078000099F90011124822B8113D1E0C15079F788
:100790008AE090E00E943C028D2FDF91CF911F9163
:1007A0000F91089580915D0390915E03009739F059
:1007B000019790935E0380935D030C94820380E025
:1007C00008958F929F92AF92BF92CF92DF92EF9255
:1007D000FF92CF93C82E60E070E0CB010E94DD0253
:1007E00081113DC080E1C89E600111248AE3C81ACE
:1007F0008EEFD80AE12CF12C12C020915D033091CC
:100800005E032115310571F02150310930935E03EB
:1008100020935D030E9482038FEFE81AF80AEC141C
:10082000FD0458F30E94D203882E912CA12CB12CE8
:100830000E94D203C82F0E94D203C82ED12CE12CD3
:10084000F12C7601DD24CC24DC2AC828D928EA281A
:10085000FB280E94D203F82A0E94A10304C0CC24E2
:10086000CA94DC2C7601B601C701CF91FF90EF90BE
:10087000DF90CF90BF90AF909F908F900895BF92E0
:10088000CF92DF92EF92FF920F931F93CF93DF935C
:10089000FC011092000148E9F42E01C0FE01EF01B5
:1008A0008991982F907F903209F4D3C028F499232E
:1008B00049F0903199F72EC0903909F474C1903FF6
:1008C00069F79EC18F70893099F028F4813049F022
:1008D000883021F70BC08B3079F060F08F30F1F663
:1008E0000DC085E08A95F1F70000D8CF5D98D6CF8E
:1008F0005D9AD4CF5E98D2CF5E9AD0CF809100011E
:100900009181A82FB0E0AD5BBD4F9C938F5F80932A
:100910000001F8C08F708530B9F180F4823009F1A0
:1009200038F4882309F45CC1813009F0B7CF17C0CF
:100930008330C9F0843009F0B1CF17C0883079F125
:1009400038F4863009F482C0873009F0A7CF1FC081
:100950008A3079F140F18B3009F0A0CF2CC0539A46
:100960009DCF5B989BCF5B9A99CF8091000199B105
:10097000E82FF0E0ED5BFD4F93FB992790F9908312
:100980008F5F809300018ACF0E942F0287CF109142
:100990000001EF01229681810E94DD01A9C0109122
:1009A000000180E003C01091000181E00E949B01E2
:1009B0009FC03180A7C0D180DD0CC280E380EF01F1
:1009C00024960E942F02109100018D2D0E94DD01BE
:1009D000E12FF0E0ED5BFD4F80831F5F109300017E
:1009E0008E01BC2EBC0C05C0F80181918F010E94C4
:1009F000DD01B012F9CFCC0DD11D0E942202EE20F4
:100A000009F44CCF0E942F02109100018D2D8160BE
:100A10000E94DD0103C080E00E949B01E12FF0E015
:100A2000ED5BFD4F80831F5F10930001EA941091EE
:100A30000001E110F0CF81E00E949B01E12FF0E086
:100A4000ED5BFD4F80831F5F109300010E94220227
:100A500025CF8F708530C1F178F4823011F130F4F8
:100A60008823D9F0813009F019CF19C08330D9F02B
:100A7000843009F013CF19C0883089F138F48630FA
:100A800009F48EC0873009F009CF21C08A30C9F13E
:100A900050F18B3009F002CF38C02798FFCE279A4B
:100AA000FDCE2F98FBCE2F9AF9CE9091000183B105
:100AB000E92FF0E0ED5BFD4F881F8827881F8083BA
:100AC0009F5F90930001EACE0E948E01E7CE1091C5
:100AD0000001EF01229681810E943C0109C0109122
:100AE000000180E003C01091000181E00E94FA0043
:100AF000E12FF0E0ED5BFD4F80831F5F109300015D
:100B0000CDCE4180EF012296C9CED180DD0CC280CE
:100B1000E380EF0124960E948E01109100018D2D3B
:100B20000E943C01E12FF0E0ED5BFD4F80831F5FF1
:100B3000109300018E01BC2EBC0C05C0F801819100
:100B40008F010E943C01B012F9CFCC0DD11D0E9443
:100B50008101EE2009F4A2CE0E948E0110910001C5
:100B60008D2D81600E943C0103C080E00E94FA004C
:100B7000E12FF0E0ED5BFD4F80831F5F10930001DC
:100B8000EA9410910001E110F0CF81E00E94FA0098
:100B9000E12FF0E0ED5BFD4F80831F5F10930001BC
:100BA0000E9481017BCE8F708130A9F020F08230CD
:100BB00009F074CE17C05298539A81818093C50072
:100BC00082818093C400F092C10083818093C2002F
:100BD000EF01249663CE1092C1005A9852985B9808
:100BE00053985CCE91813296892FDF0103C02D91FD
:100BF0002093C6008150D8F7EF01C90FD11D4ECE0A
:100C0000DF91CF911F910F91FF90EF90DF90CF90E8
:100C1000BF900895E8EBF1E0A3E4B2E094919D93D6
:100C2000319691E0EB3CF907C9F76770685F609314
:100C3000480280934E0283E492E00C943F041F929A
:100C40000F920FB60F9211240F900FBE0F901F90AE
:100C500018951F920F920FB60F9211240F900FBE8E
:100C60000F901F9018951F920F920FB60F9211249C
:100C70008F939F93EF93FF93CF93DF931F92CDB703
:100C8000DEB78091C6008983809142018F5F8F73A8
:100C900090914101981741F0E82FF0E09981EF5FC2
:100CA000FE4F9083809342010F90DF91CF91FF918F
:100CB000EF919F918F910F900FBE0F901F901895FD
:100CC000CF93DF9300D000D0CDB7DEB780E880931C
:100CD0006100109261008FEF80936600559A8BB18E
:100CE00090E289278BB9579A5F9A2FEF81EE94E0B3
:100CF000215080409040E1F700C00000E8E6F0E0BD
:100D0000A3E4B2E084918D93319620E0E83BF207B2
:100D1000C9F783E492E00E943F0410E0612F80E075
:100D20000E940A061F5F1830C9F78FE39CE90197FC
:100D3000F1F700C000008AB180668AB95D9A8BB174
:100D40008C7F8BB98AB18C7F8AB95298539A5B9AFF
:100D5000279A2F9AFAE03F2EEFE3FCE93197F1F75B
:100D600000C0000010E0612F80E00E940A061F5FB3
:100D70001830C9F760E08AEA0E940A0664E08AEA4D
:100D80000E940A06419A399A10E03C9A3D9887B130
:100D9000807F87B988B18F6288B987B18F6287B940
:100DA000FFEF23EC89E0F15020408040E1F700C0E4
:100DB00000008AE4449A44988150E1F740E050E012
:100DC00060E070E080E40E94810288E090E00E9490
:100DD0003C024AEA51E060E070E088E40E9481024F
:100DE0000E94BC0287FF08C01F5FEFE3FCE9319758
:100DF000F1F700C00000C9CF82E090E00E943C0201
:100E00000E94BC02813009F0EAC10E94BC028A3A09
:100E100009F0E5C182E090E00E943C0260E082E0DF
:100E20000E940A0640E050E060E070E087E70E9420
:100E3000810280E190E00E943C0240E050E060E3EB
:100E400070E589E60E9481020E94BC0287FDC7C14D
:100E50000E94BC02082F809343030E94BC020E94A0
:100E6000BC020E94BC020E94BC020E94BC028AE03A
:100E700090E00E943C0207FD11C08FE39CE90197BE
:100E8000F1F700C000001A3008F0A9C1EFE3FCE957
:100E90003197F1F700C000001F5FC4CF06FB0027A9
:100EA00000F90093430360E083E00E940A0640E0FB
:100EB00050E060E070E082E40E9481020E94BC0287
:100EC0000E94BC020E94BC020E94BC020E94BC02A2
:100ED0000E94BC0288E290E00E943C0240E050E0A8
:100EE00060E070E083E40E9481020E94BC020E94E4
:100EF000BC02182F0E94BC02412F50E060E070E05D
:100F0000762F652F542F4427482B4093440350934A
:100F10004503609346037093470384E190E00E9489
:100F20003C0260E084E00E940A06609144037091F4
:100F3000450340E050E089E40E9481020E94BC0227
:100F40000E94BC020E94BC020E94BC020E94BC0221
:100F50000E94BC020E94BC0288E290E00E943C0217
:100F600040E050E060E070E08CE40E94810280E8A4
:100F700090E00E943C0260E085E00E940A06009139
:100F800044031091450340E050E0B80187E40E941B
:100F900081020E94BC020E94BC020E94BC020E940C
:100FA000BC020E94BC020E94BC020E94BC0284E1FE
:100FB00090E00E943C0240E050E0B80187E70E94C8
:100FC00081020E94BC020E94BC020E94BC020E94DC
:100FD000BC020E94BC020E94BC020E94BC0284E1CE
:100FE00090E00E943C0242E050E060E070E086E465
:100FF0000E9481020AE010E00E94BC020150110927
:10100000D9F784E690E00E943C0260E086E00E940E
:101010000A06609144037091450340E050E087E781
:101020000E94810280E290E00E943C0240E050E099
:1010300060E070E083E70E9481020E94BC020E948F
:10104000BC020E94BC020E94BC020E944A0200E252
:1010500010E00E94820301501109D9F78AE090E064
:101060000E943C0260E087EA0E940A0640E052E0EB
:1010700060E070E080E50E9481020E94BC020E9454
:10108000BC020E94BC020E94BC02182F84E190E0C6
:101090000E943C02193039F08FE39CE90197F1F787
:1010A00000C00000E3CF60E088E00E940A068AE00A
:1010B00090E00E943C0241EF5FEF6FEF70E886E442
:1010C0000E9481020E94BC020E94BC020E94BC02DB
:1010D0000E94BC020E94BC020E94BC020E944A0202
:1010E00009E410E00E94820301501109D9F78AE057
:1010F00090E00E943C02609144037091450340E0FF
:1011000050E087E70E94810280E290E00E943C026A
:1011100040E050E060E070E08DE40E9481020E94B7
:10112000BC020E94BC020E94BC020E94BC020E943F
:101130004A0209E410E00E94820301501109D9F724
:1011400080E092E00E943C0240E050E060E070E00D
:101150008CE40E9481028AE090E00E943C0280E0E0
:1011600092E00E943C0260E089E00E940A066091E1
:1011700044037091450340E050E087E70E948102FC
:101180000E94BC020E94BC020E94BC020E94BC02DF
:101190000E94BC020E94BC020E94BC0284E190E05A
:1011A0000E943C0240E050E060E070E08AE60E946D
:1011B00081020E94BC020E94BC020E94BC020E94EA
:1011C000BC020E94BC020E94BC020E94BC0284E1DC
:1011D00090E00E943C028AEF90E00E943C0260E0B6
:1011E00080E10E940A0664E080E10E940A0680E035
:1011F0000E94E10380E00E94E10381E00E94E1039C
:1012000082E00E94E10383E00E94E10381E00E940A
:10121000E1036B017C01DC01CB010197A109B1095C
:1012200060E08E3F9F4FAF4FBF4F20F08AE10E949A
:101230000A0659CD80EF0E940A0661E080EF0E9405
:101240000A0662E080EF0E940A0663E080EF0E94D7
:101250000A06569A8BB190E489278BB9FA82E98203
:1012600000E012E001C0B92C8FE19EE40197F1F794
:1012700000C00000C701B6010E94DD020E94D20337
:10128000A82E63E4862E61E0962E0E94D203F4011C
:1012900081934F01F3E48F16F2E09F06B1F72AEA3B
:1012A000A21621F00E94A1039B2CDDCF9B2C9394CE
:1012B00067E08B2D0E940A060E94A1038111D3CF03
:1012C00083E491E00E943F048AE090E00E943C02A7
:1012D000A60169817A8188E50E9481028FE090E011
:1012E0000E943C028AB18F608AB980EF0E944F034E
:1012F0000E94CC0210935E0300935D038BEB0E946F
:10130000720323E432E009C0F90181919F01EB836C
:101310003C830E9472033C812B81590183E492E05B
:10132000A81AB90A8091000190E0A816B90660F3E6
:1013300006C08FEF0E9472039FEFA91AB90AEFEF60
:10134000AE16E1E0BE06A8F308C0019790935E03D5
:1013500080935D038FEF0E94720380915D039091F3
:101360005E03009791F71092590358E0B52E0E9442
:101370001403A82E0E941403F0E1AF9E90011124E3
:10138000822B0E944F03BA9491F78FE00E944F0383
:101390008AE090E00E943C0287B1807F87B92FEFFE
:1013A00089EF90E0215080409040E1F700C00000BC
:0613B0005ACFF894FFCFB4
:00000001FF
